:020000040000FA
:020000000528D1
:080008000528383083008B014C
:100010008B1B07288430810010308500003086005B
:100020008312FE30850086018E018F0181309000A1
:10003000930194019501CA2883161030850086012A
:100040008312FE308500860111229D211308940041
:100050009301851405118511051E93140515051EC0
:1000600093158510051E13158515051E131705110B
:10007000051E13168514051E93161308031D42282A
:100080009501262814020319472895014D28950A41
:100090001508363C031826289503931C6B28901FDF
:1000A0005C280F181C280430101C10308E070E0816
:1000B0003C3C031C8E01CA28100C0F39203E8400E2
:1000C0000130101C103080070F18692801308F0094
:1000D0001C28E4212628131D7E28900A1008823C43
:1000E000031D742890017A281008103C031D7A28FB
:1000F00080309000F0213C3040222628931D9A2821
:10010000901F8D280F181C280430101C10308E02F0
:100110000318CA283C308E00CA28100C0F39203E24
:1001200084000130101C103080020F186928013043
:100130008F001C28131EAA2890037F301002031D75
:10014000A4280F3090007A28100A031D7A288130E5
:1001500090007A28931EC828203084000E089A0048
:10016000FB2000089B00840A00089C00840A1A08EF
:1001700031219A0A0408283C031DB12817210430B4
:100180008F00E520FF3903191C2810308F001C2830
:10019000131FE428203084000E089A001A086C21EE
:1001A00016088000840A17088000840A9A0A040846
:1001B000283C031DCE2802308F00E520FF390319AB
:1001C0001C2808308F001C281C28203084000E08B2
:1001D0009A001A086C2116080002031DFF34840AD5
:1001E00017080002031DFF34840A9A0A0408283CF9
:1001F000031DE928003486010E308500861705149A
:10020000061706130510061706130617061305141E
:100210000617061306170613061706130617061306
:100220000617061306170613051086130800860125
:100230000E308500861705140617061305100617DD
:1002400006130617061306170613061706130617D6
:10025000061306170613061706130617061386134A
:1002600008009D0086010E308500861705140617CC
:100270000613051006170613051406170613063095
:100280009E0005109D1A05149D0D061706139E036A
:10029000031D412908309E0005109B1B05149B0D72
:1002A000061706139E03031D4C2908309E000510F7
:1002B0009C1B05149C0D061706139E03031D57294E
:1002C00005108613861750309E00051A6A299E0372
:1002D000031D652986130800980086010E308500ED
:1002E00086170514061706130617061305100617BA
:1002F0000613063099000510981A0514980D061774
:1003000006139903031D7B29051008309900061771
:100310000613960D1610051A16149903031D872946
:100320000830990006170613970D1710051A1714B1
:100330009903031D9229861308004A22803029223E
:100340000E08F9210F08031DAE2920302C22203081
:100350002C2220302C2220302C22E4290F1CB929F9
:100360002A302C2220302C2220302C2220302C220B
:10037000E4298F1CC42952302C2245302C224F30C6
:100380002C224B302C22E4290F1DCF2957302C2250
:1003900052302C224F302C224B302C22E4298F1D3E
:1003A000DA2952302C2245302C2252302C22523065
:1003B0002C22E4290F1EE42957302C2245302C2210
:1003C00052302C2252302C224A22C0302922203096
:1003D00084000008F921840A0408283C031DE92947
:1003E000901FF5291008452208001008C038452242
:1003F00008009100110E0F39303E9200393C03186D
:10040000032A2730920712082C2211080F39303E98
:100410009200393C03180E2A2730920712082C222A
:100420000800CD30402203303C220A3040223330D5
:10043000292202303C22283029220830292201308A
:10044000292203304022063029220C30292286013D
:1004500008008C0000302E2A8C00103086000C0E14
:100460000F39860486168612103086050C080F395F
:1004700086048616861208008C0000308600362A14
:100480008D008D03031D412A080029220F302922E7
:0A049000860108000C302922080044
:00000001FF
